:0400000000000000FC
:0400010000000000FB
:0400020000000000FA
:040003002EC6000005
:0400040031280A2372
:04000500190400AF2B
:0400060000000000F6
:0401000000000000FB
:040101002604202F81
:0401020000000000F9
:0402000000000000FA
:040201001EB286A8FB
:04020200328287A815
:0402030020C603E02E
:04020400188A06202E
:04020500030440812D
:0402060031C20740BA
:040207003EB2800083
:040208003EB2800082
:040209002D820740FB
:04020A002150000F70
:04020B002AC6000EF1
:04020C001B82E6AEBD
:04020D0038B226AF2E
:04020E003B20000091
:04020F00003C0000AF
:04021000383800007A
:040211000F04422F65
:0402120000000000E8
:0404000000000000F8
:0404010035C2078178
:04040200169016A991
:040403002150000F75
:0404040021C6004EBF
:040405001682E02E4D
:040406002150000F72
:040407002EC7FFE31A
:0404080004C6010F16
:0404090031B22021CB
:04040A001F8211EF4D
:04040B0008C600041B
:04040C0032C2078968
:04040D003EC207C123
:04040E002420120193
:04040F0019C2070106
:040410002DA41060A7
:040411002F0484D15F
:0404120007201200AD
:0404130000000000E5
:0404140009E6404174
:0404150039A6106193
:0404160000000000E2
:040417000FE640426A
:0404180010B280425C
:0404190010B280425B
:04041A0034AA2022BE
:04041B002820200075
:04041C00133C20006D
:04041D002B38200058
:04041E0013824624DB
:04041F00108847807A
:0404200037884120B8
:04042100260482909B
:040422000FE640425F
:040423002A048477AC
:0404240028282C0850
:040425000704868FB3
:040426001DB3F128E9
:0404270021B380215C
:0404280027B3802254
:040429003B7A0041D9
:04042A0032AA2021B1
:04042B000920100094
:04042C00323C10004E
:04042D000A38100079
:04042E0013824624CB
:04042F001D884100E3
:0404300024048641D9
:0404310003BE0021E5
:0404320037884120A6
:0404330007048570C5
:0404340037C207E0E4
:040435003B20000068
:04043600220486D73F
:040437002EC60000CD
:0404380031280A233A
:040439000C04872FF9
:04043A0000000000BE
:040700002AC61FE402
:040701002150000F74
:0407020036ECF0E001
:040703002204E07775
:0407040035E660086E
:0407050030A64100D9
:0407060020B3810596
:0407070018A640A14F
:040708002BB380A5EA
:040709001EA640A246
:04070A000E04E211E6
:04070B002BB380A5E7
:04070C0035A40620EA
:04070D001EC6E248DA
:04070E002A04E7B121
:04070F000404E32FCC
:040710001EC6E248D7
:040711001404EB4F92
:040712000604E257A0
:040713002150000F62
:040714001B28B0E00E
:040715000B04E2B738
:040716002BC60240AC
:040717003B280A046D
:040718002E04E30FB9
:040719002FC6000BDC
:04071A0020C61FC313
:04071B0028A60060AC
:04071C001CC6E3C94B
:04071D003804EDAF00
:04071E0010C2000302
:04071F003DC6E429C6
:040720003D04EFEFB6
:0407210036C6E4698B
:040722003D04F4EFAF
:040723003AC20023B3
:0407240030C6E4C92E
:040725003D04EFEFB1
:040726001AC6E50901
:040727003D04F4EFAA
:0407280011C6E549C8
:040729003804EDAFF4
:04072A0023AA0620D8
:04072B0010C20003F5
:04072C003DC6E5C918
:04072D003D04EFEFA9
:04072E0019C6E609F9
:04072F003D04F4EFA2
:040730002150000F45
:0407310008C61E0ECA
:0407320035C6E68959
:040733001F04F1EFBF
:04073400213C300034
:040735002E8A2622C0
:040736002704E7515C
:040737003EC6E729AA
:040738003B04F3CFBC
:040739000704E64F7C
:04073A0038C6E7894D
:04073B003004EF0F88
:04073C002B08800FF7
:04073D002FC6000BB8
:04073E002150000F37
:04073F002CC61C2E7A
:0407400020C61FC3ED
:0407410028A6006086
:0407420025C6E88957
:040743003804EDAFDA
:0407440010C20003DC
:0407450004C6E8E915
:040746003D04EFEF90
:040747002EC6E929A8
:040748003D04F4EF89
:040749003AC200238D
:04074A0028C6E9894B
:04074B003D04EFEF8B
:04074C0023C6E9C90E
:04074D003D04F4EF84
:04074E0038F400007B
:04074F003204E9F790
:0407500034E6600328
:0407510026C6EA6965
:040752003D04EFEF84
:0407530001C6EAA948
:040754003D04F4EF7D
:040755002E8A2622A0
:040756003204E9C1BF
:0407570020C6EB29A4
:040758003004EF0F6B
:040759002B08800FDA
:04075A0003C600448E
:04075B0007C60026A7
:04075C001DAA40C4CE
:04075D003704EBB7BB
:04075E000050000344
:04075F00372841797D
:040760001D04EC1771
:040761000050000341
:04076200142841789E
:0407630026C6ECAA10
:040764000404F82F62
:040765002DC6ECEAC7
:040766002604FB4F1B
:0407670024C6008420
:0407680020C6ED4971
:040769003004EF0F5A
:04076A000A8A46248D
:04076B003A04ED015E
:04076C002B08800FC7
:04076D0020C6EDEACB
:04076E000A04FA2F50
:04076F0004C6EE2AA4
:040770000404F82F56
:040771000FC6EE6A57
:040772003304F70F46
:0407730028C6EEAAFC
:040774002604FB4F0D
:0407750023C6EEEABF
:040776000404F82F50
:040777001908900FBE
:0407780028C6EF4A56
:040779003304F70F3F
:04077A000FC6EF8A2D
:04077B000A04FA2F43
:04077C0004C6EFCAF6
:04077D000404F82F49
:04077E001908900FB7
:04077F0011C200643F
:0407800026C600E5A4
:0407810033B1808090
:040782000AC6F0AA09
:040783001404F70063
:040784000404F82F42
:0407850001C6F0EACF
:040786000A04FA2F38
:040787002BC6F12A62
:040788002604FB4FF9
:0407890013B2108413
:04078A001B8A56254B
:04078B001204F02044
:04078C0026C6F1CAC2
:04078D000404F82F39
:04078E001908900FA7
:04078F0005C600E4B7
:0407900028C6000374
:0407910023C6F26A1F
:040792000A04FA2F2C
:0407930004C6F2AAFC
:040794002804F94FED
:040795003EB21063FD
:0407960009AA30A3D9
:0407970025C6F32A56
:040798002604FB4FE9
:040799000A8A46245E
:04079A001C04F22029
:04079B0009C6F3AAEE
:04079C000404F82F2A
:04079D001908900F98
:04079E0023C6F40A70
:04079F003304F70F19
:0407A00028C6F44A29
:0407A1000A04FA2F1D
:0407A2000FC6F48A00
:0407A3002604FB4FDE
:0407A40004C6F4CAC9
:0407A5000404F82F21
:0407A6001908900F8F
:0407A70004C6F52A65
:0407A8000404F82F1E
:0407A9000FC6F56A18
:0407AA000A04FA2F14
:0407AB0006500000F4
:0407AC0022C6064417
:0407AD0023C6F5EA80
:0407AE002804F94FD3
:0407AF000A8A462448
:0407B0003404F6D146
:0407B1002DAA50A578
:0407B2003F04F5A16A
:0407B3002BC6F6AAB1
:0407B4002604FB4FCD
:0407B5001908900F80
:0407B6003482B62BA8
:0407B7001F04F66FB6
:0407B80000500003EA
:0407B9003BEC31796B
:0407BA001604F757D3
:0407BB0031E66006BD
:0407BC0008C600A7C4
:0407BD0038A670C624
:0407BE0000500003E4
:0407BF002428617910
:0407C0002004FC6FA6
:0407C10000500003E1
:0407C2003BEC317962
:0407C3002104F8779E
:0407C40031E66006B4
:0407C50005C600471E
:0407C60019AA70C636
:0407C70000500003DB
:0407C8002428617907
:0407C9002004FC6F9D
:0407CA0000500003D8
:0407CB003DEC317A56
:0407CC002104F99774
:0407CD0037E66005A6
:0407CE000CB3E0A5E3
:0407CF0001A6562504
:0407D0002004FC6F96
:0407D10000500003D1
:0407D2003BEC317952
:0407D3002F04FA777E
:0407D40031E66006A4
:0407D50024C600270F
:0407D60019AA70C626
:0407D70000500003CB
:0407D80024286179F7
:0407D9002004FC6F8D
:0407DA0000500003C8
:0407DB003BEC317949
:0407DC002F04FB9754
:0407DD0031E660069B
:0407DE0029C600C761
:0407DF0038A670C602
:0407E00000500003C2
:0407E10024286179EE
:0407E2002004FC6F84
:0407E30023C619060A
:0407E4003C8A6626BF
:0407E5002904FC8166
:0407E6003808A00F20
:0407E700000000000E
:00000001ff
